:020000040000FA
:0600000034EF15F01200C0
:0608000034EF15F01200B8
:0608080069EF13F012007D
:06081800DFEF13F01200F7
:06082A000100942A000009
:08083000600000007C000000E4
:0808380021EC08F00001010EA3
:10084000FA6FFB6FFC6F330EF06FE66A5FDBE55209
:10085000080E0001F16FF26BF36BF46BF56BF66B46
:100860001200D9CFE6FFE1CFD9FF080EE126060E30
:100870000101C85D03E36D50020B12E00001F307B4
:10088000000EF45B0001F351F41109E10001F107DE
:10089000000EF25B0001F151F21101E1FF008DD178
:1008A0000001FA51040A01E164D1070A01E11CD1F7
:1008B000010A1DE0030A01E07CD1EFC0E6FF010E52
:1008C000E66E4CDBE552E552010EE66EF70EE66E83
:1008D000000EE66E1FEC0FF0E552E552E5520009FE
:1008E00005E0F7C0F8F00001020EFA6F66D10201D0
:1008F000D25101E0F8D0FF0E0001F85D07E140DBC6
:10090000000903E00001010EFA6FEDD0FE0E0001B8
:10091000F85D07E145DB000903E00001010EFA6F15
:10092000E2D0800E0001F85D06E10001F96B0001E4
:10093000030EFA6FD8D0810E0001F85D31E1EFC0EF
:10094000E6FFE66A0BDBE552E552000EE66E020EAC
:10095000E66E000EE66E010EE66E08EC0AF0E55259
:10096000E552E552E552E76E070EE7CFDBFF070ED3
:10097000DB040BE1EFC0E6FF010EE66EEFDAE552B5
:10098000E5520001040EFA6F0AD0EFC0E6FF010E37
:10099000E66EE4DAE552E5520001010EFA6FA3D0EB
:1009A000820E0001F85D11E10001010EEF6FEFC052
:1009B000E6FF020EE66ED2DAE552E5522FDB0009C1
:1009C00003E00001010EFA6F8ED0830E0001F85D86
:1009D00010E10001EF6BEFC0E6FF020EE66EBEDA3B
:1009E000E552E5521BDB000903E00001010EFA6F3E
:1009F0007AD0800E0001F85D55E2030E0001F81573
:100A0000E76E010EE7CFDBFF0C0E0001F815E840A2
:100A1000E8403F0BE76E020EE7CFDBFF020EDB5034
:100A2000030805E1020EF36E020EF3CFDBFF300E7A
:100A30000001F815E8380F0B010FE76E030EE7CF42
:100A4000DBFF030EDB50030805E1040EF36E030E1B
:100A5000F3CFDBFF060E146E400E0001F81514C034
:100A6000E7FFE75204E0E8427F0BE706FCE1E76EB0
:100A7000040EE7CFDBFF040EDBCFE6FF020EDBCF79
:100A8000E6FF010EDBCFE6FF030EDBCFE6FFFAD871
:100A9000E552E552E552E552000903E00001010E7E
:100AA000FA6F21D0DF6A0E0EDF5C1AE2DF50EA6ACD
:100AB000CE0FE96E000EEA22EF500001F85D0EE164
:100AC000EFC0E6FFE66A4ADAE552E552DFCFE6FF1D
:100AD000150EE66E8EEC0CF0E552E552DF2AE3D7F8
:100AE0000001010EFA6F69D0EFC0E6FFE66A36DA60
:100AF000E552E552000EE66E020EE66E000EE66E60
:100B0000010EE66E28DBE552E552E552E552050E90
:100B1000F3CFDBFF060EF4CFDBFFD950050FE96EF4
:100B2000DACFEAFFEE50ED1023E0D950050FE96E61
:100B3000DACFEAFF000ED880EE54800EED540EE2BC
:100B4000000EE66E020EE66E000EE66E010EE66E1A
:100B500025EC0DF0E552E552E552E5520001010E9B
:100B6000FA6FEFC0E6FF010EE66EF8D9E552E552E6
:100B700024D0EFC0E6FFE66AF1D9E552E552000E57
:100B8000E66E020EE66E000EE66E010EE66EBBDB52
:100B9000E552E552E552E55200090AE00001010E76
:100BA000FA6FEFC0E6FF010EE66ED8D9E552E552C6
:100BB00004D00001010EFA6F00D0080EE15C02E2E1
:100BC000E16AE552E16EE552E7CFD9FF120072EC1F
:100BD0000BF0EFC0E6FFE66AC1D9E552E552F0C07E
:100BE00081FF140EE66E95DAE552FE0EDB500B0D1A
:100BF000F3CFECF00001F35095EC0BF0EECFEDF0FD
:100C0000EDCFEEF0F32895EC0BF0EECFE2F0EDCF68
:100C1000E3F0020EF32495EC0BF0EECFE4F0EDCF11
:100C2000E5F0030EEC27DE6BDF6BE06BE16BDD6B59
:100C3000F28C0AEC0CF0BD6A050EBD6E9E6AF28E57
:100C4000DDA5FED7F29E330E816EDDB303D0E4EC5A
:100C50000BF016D0EA51E65DEB51E7590BE2E85193
:100C6000E91104E0E807000EE95B04D0E4EC0BF0C6
:100C7000EA6BEB6BEA51E65DE66FEB51E759E76F24
:100C800077EF0BF072EC0BF0410EE1263B0EDB6AC6
:100C9000360EDB6A030EF36E370EF3CFDBFF020E68
:100CA000F36E380EF3CFDBFF010EF36E390EF3CF88
:100CB000DBFFFD0EDBA003D03C0EDB6A05D0030E8C
:100CC000F36E3C0EF3CFDBFFFD0EDBA202D0040E71
:100CD00001D0030EF36E3D0EF3CFDBFF0001FB519D
:100CE000060A01E1EDD0030A01E1DBD0010A01E1CE
:100CF000C1D0070A01E1B1D0010A6CE0030A01E0AA
:100D0000E6D00201C86B180EC85D06E266EC0BF077
:100D1000EE6AED6AC82BF7D7400EDB6AFE0EDB5099
:100D2000F36E400E30EC0CF050E23C0EDB50E76E00
:100D30003E0EE7CFDBFF3D0EDB50F36E3E0E30EC98
:100D40000CF040E2D950360F146EDACF15F03E0E9B
:100D5000DB500F011424C6EC0BF0C7D8E552FC0E93
:100D6000DB50020819E13F0EDB6ADB50010827E384
:100D70003F0EDBCFE6FFCAD8E5523EEC0BF0D8A021
:100D800002D040EC0CF0D9CF14F0DACF15F028ECFB
:100D90000CF03F0EDB2AE9D73F0EDB6AFC0EDB507E
:100DA000030805E0FC0EDBCFE6FFB0D8E5523EECD1
:100DB0000BF0D8A002D040EC0CF028EC0CF03E0E6A
:100DC000DB2AB9D7400EDB2AA9D70201C86B180E5F
:100DD000C96F73D0FD0EDBA00CD0520EF36E300E37
:100DE000F3CFDBFF470EF36E310EF3CFDBFF420E86
:100DF0000BD05F0EF36E300EF3CFDBFF5F0EF36EA2
:100E0000310EF3CFDBFF5F0EF36E320EF3CFDBFF5D
:100E1000FD0EDBA202D0570E01D05F0EF36E330E33
:100E2000F3CFDBFFFC0E35EC0CF0340EE7CFDBFF2D
:100E30003A0EF36E350EF3CFDBFF0201D2510DE116
:100E40000201D950300FD36FDACFD4F20201060E6F
:100E5000D76F80EC0BF00001FB2B0201D25139E17E
:100E600002018D0ED36F2A0ED46F0201060ECDEC57
:100E70000BF023D0D9CF14F0DACF15F0020166ECD5
:100E80000BF0EECFE6FFEFCFE6FF00D9E552E552DB
:100E9000000902E00201C82B0201C951C85D19E333
:100EA0000CD00201D25115E102018A0ED36F2A0E35
:100EB000D46F0201020ECDEC0BF00001FB2B09D028
:100EC000010EFB6FF36E3B0EF3CFDBFF02D0010E82
:100ED000FB6F3B0EDB50146E410EE15C02E2E16AF7
:100EE000E552E16E145077EF0BF072EC0BF0FE0E52
:100EF000DBA003D00001F08D02D00001F09DDBA249
:100F000002D0F08F01D0F09F77EF0BF0EBDB040EF7
:100F1000E126D9CFE6FFDACFE6FF3FDAE552E55228
:100F2000020EDB50E76E030EE7CFDBFFFE0EDB5059
:100F300004E1030EDB50020803E0030EDB5004E182
:100F40000001F081F09903D00001F091F089040EC6
:100F5000E15C02E2E16AE552E16EC9D3C3DBFE0E59
:100F6000DB50020803E0FE0EDBCFCAF2FD0EDB50C1
:100F700003E00201CA5102E1829001D08280B7D31E
:100F800046EC0CF00AE10201820ED36F2A0ED46FF8
:100F90000201070ECDEC0BF0DF6EDF50E552A7D358
:100FA000A1DB0C0EE126DF6AD950090FE66E000EB8
:100FB000DA20E66EF2D9E552E552DE52760EDD6EAB
:100FC000090E35EC0CF0020EE7CFDBFF2E0EF36EB0
:100FD000030EF3CFDBFF0A0EEBEC0BF02E0EF36EDD
:100FE000050EF3CFDBFF0B0EF0EC0BF00D0E14EC47
:100FF0000CF00A0E0FEC0CF00201D25105E1D4DB2B
:10100000080ED76F7DDBDF6EDF50146E0C0EE15CD7
:1010100002E2E16AE552E16E145069D346EC0CF04D
:101020000DE10201800ED36F2A0ED46F0201010E72
:10103000D76F0201D86F0201D26FDF6EDF50E55229
:1010400056D3806A826A330E816E92680C0E936E5C
:10105000FE0E946ED06A400EF26E800EF16E050E9A
:101060009D6ECD6ABD6ECA6E0F0EBA6E0001010E86
:10107000EF6F1200110ECB6E090EBB6E040ECA6E1E
:101080000F0EBA6E0001DC6B949212002BDB090E7E
:10109000E126DF6AFE0EDB50E76E070EE7CFDBFFCF
:1010A000640E17DB09C0DBFFE0DB010EE7CFDBFFDF
:1010B000640E0FDB2BDB020EDCDBD7DB030EE7CF8E
:1010C000DBFFFD0EDBCF14F0FE0EDBCF15F00001D1
:1010D000156A070E14C0DBFF640EFBDA09C0DBFFE4
:1010E0007ADB640EF6DA12DB050EC3DB79DB020174
:1010F000D25105E159DB060ED76F02DBDF6EDF5000
:10110000146E090EE15C02E2E16AE552E16E1450F0
:10111000EED2E8DA020EE126DF6AFE0EDB50DF5C7B
:1011200013E2010EDB6ADF50146E156AD890155079
:1011300004E6FA0E145C000E155804E2DF2ADF06FE
:10114000DF2AF1D7DF2AE9D7020EE15C02E2E16A89
:10115000E552E16ECCD2C6DA450EE126DE6ADD6AE2
:101160000001F95107E1010EF96F0201CB6BCC6B65
:10117000CD6BCE6B400EE66ED950050FE66E000EBD
:10118000DA20E66E1FEC0FF0E552E552E552000959
:1011900001E19AD00201CD6BCE6B030EDB6A020E29
:1011A000D1C2DBFF020EDB50F36E030E59DB01E30D
:1011B0009BD0D9CFE9FFDACFEAFFEE50ED1001E086
:1011C00093D0C80ECB5D000ECC5916E2D950050F56
:1011D000146EDACF15F0030EDB500F011424D6DAAB
:1011E000FD0EDB500201CB250F01E96EFE0EDB5038
:1011F0000201CC210F0117D0D950050F166E030E36
:10120000DB500F011624C2DACBC214F0CCC215F0A9
:10121000C80E145E000E155AFB0EDB501424E96E46
:10122000FC0EDB501520EA6EE552E750EF6E02012E
:10123000CB2B000ECC23900ECB5D010ECC5905E3D9
:10124000000ECB25146E400E38D0080ECB5D000E7C
:10125000CC5937E327DB500803E024DB600806E1C4
:101260000C0ECB5D000ECC592CE323D0040EFFD91D
:10127000EFCF18F0060EFBD9EF501824166E176A40
:10128000000E1722040E086E096A16C00DF017C072
:101290000EF0D9EC14F006C014F007C015F0080EDB
:1012A0001426000E152202011450CB5D1550CC59A6
:1012B00008E3000ECB25146E800ECC2114C0DEFF97
:1012C000DD6E030EDB2A6ED70201CD2B000ECE237E
:1012D000CD1D0AE1CE1D08E1000ECB25146E200EB7
:1012E000CC2114C0DEFFDD6EDECF14F0DDCF15F0B3
:1012F00014C0F3FF15C0F4FF450EE15C02E2E16AA1
:10130000E552E16EF4D1EED9E652DF6A0001FC51FC
:10131000030A2EE0010A17E0030A3AE1040E086E00
:10132000096A04C10DF005C10EF0D9EC14F006C035
:10133000CFF207C0D0F2080E0201CF27000ED02353
:101340000001FC2B27D00201D25112E10201C80E8C
:10135000D880CF55000ED05504E347DA9DDAFC6FF4
:1013600007D043DA0201C80ED76FCAD90001FC2B9F
:101370000201D2510FE10201C80ECF5F000ED05B17
:10138000FB0EDBCFD3F2FC0EDBCFD4F285DA01D03B
:10139000010EFC6FDF50E552AAD1A4D9030EE1265D
:1013A000DF6A010EDB6A200EF36E020EF3CFDBFF65
:1013B000D6D90800F550E66E3CDAE552E750EF6EFC
:1013C000CED9F62A19DA010E71DAEF6EC8D9F626EF
:1013D00013DA020E6BDAEF6E2CDAEF50FF0802E13F
:1013E00028DAEF6A5FDAFF0803E1010E40D9EF6AFD
:1013F000020E3DD9EF50FF0804E1020E38D9020E6B
:10140000EF6E030EE15C02E2E16AE552E16E6FD13C
:1014100069D90E0EE126040EDB6A070EDB6A050EA3
:10142000DB68040EFCD9DE68DD68020EDB6A030EA1
:10143000DB6A0B0EDB6A0C0EDB6A0D0EDB6AF9D978
:10144000EE6AED6A020E13D96D0EEE6EED6A040EB1
:101450000ED9EE6AED6A060E0AD9EE6AED6A010E41
:10146000E66E54DDE552F0C081FFBD6A050EBD6E2B
:10147000D1D9010ECA6ECC6A4F0ECB6E050ECA6E64
:101480009E6A070EDB5001E0D6D09EB215D09EA416
:10149000FCD79EA003D0DE68DD680AD0BF50166E70
:1014A000176A176E166ABE50AED914C0DEFFDD6E25
:1014B000B1D99E949E90E9D79E92CF50166E176A2E
:1014C000176E166ACE509FD9020E14C0DBFF030EB2
:1014D00015C0DBFF9EA004D0020EDB68030EDB68A4
:1014E000DECF14F0DDCF15F0780E145C020E155827
:1014F00011E2020EDBCF16F0030EDBCF17F0780EF1
:10150000165C020E175806E2010EF36E060EF3CFBC
:10151000DBFF02D0060EDB6A050EDB50FF081DE183
:10152000060EDB0401E179D0D9500B0FE96EDACF5A
:10153000EAFFEE2A000EEE22EE22D9500B0FE96EE2
:10154000DACFEAFFE868EE189CE1E868EE1899E166
:10155000050EEE1896E1020E5CD0050EDB50F36E20
:10156000060EDB50F35C1BE1090EDB2A0A0E01E3D9
:10157000DB2AD950090FE96EDACFEAFFFF0EEE1829
:1015800001E07FD7080EED1801E07BD7010E4CD9A2
:10159000B2D802E2EDD801D0D2D80ED972D7ABD8EA
:1015A00002E2E6D801D0CBD807D9080EDB50146E82
:1015B000156AC70E14182FE115502DE19CD824E3AD
:1015C000FB0EDBCF16F0FC0EDBCF17F0080EDB5066
:1015D0009C0F020D1650F324E96E1750F420EA6EAA
:1015E000EECF14F0EFCF15F0000E145C020E15587C
:1015F0000BE2020E146E080EDBCFE7FF1450E75E1D
:10160000080EE7CFDBFFDAD776D802E2C70E07D99C
:10161000010E0AD936D7080EDB2A010EF36E090E29
:10162000F3CFDBFF0A0EDB6A060EDB50E76E050E1A
:10163000E7CFDBFF26D7080EDB50FD0FFE0BE8429D
:10164000E66E040E33D9EE6EED6A330E816E070E30
:10165000DB50E76E040EE7CFDBFFDB50146E0E0E9F
:10166000E15C02E2E16AE552E16E145040D0E76EBF
:10167000E0D8E750E926000EEA221200FB0EDBCF8D
:10168000E6FFFE0EDB04E552E724E66EE7EC05F02C
:10169000E5523F0EDB500C0DF3CF14F03E0EDB5045
:1016A000030DF35014240201C86F020EC825C8D8D8
:1016B0000001E051EE26E151ED220201C829C0D817
:1016C0000001E651EE26E751ED221200C85120EF4D
:1016D0000CF0146E0E6E070EDBCF09F026EC15F041
:1016E000080E1200D9CFE6FFE1CFD9FF1200E55274
:1016F000E7CFD9FF1200640EF36E080E30EF0CF046
:101700000201D86B0201010ED26F120005C0DBFF8F
:101710000A0E146E0E6E080EDBCF09F026EC15F0E3
:10172000080E09C0DBFF35EF0CF0E96EEA6AD890CD
:10173000E936EA36600EE926000EEA221200FB0EB8
:10174000DBCF14F0FC0EDBCF15F0080EDB509C0F46
:10175000020D1450F324E96E1550F4201200DFCF6F
:10176000F6FF010EDBCFF7FF020EDBCFF8FF120012
:10177000080E156ADB34FE0B1536146EFD0EDB50B9
:101780001424E96EFE0EDB5015201200E96E000EE7
:10179000DA20EA6EEF50E66E1200D76F0201010EFA
:1017A000D86F0201D26F12000201D950010FD36F1E
:1017B000DACFD4F202011200EA6E090EDBCFEEFF9F
:1017C0000A0EDBCFEDFF1200E86BE96BE66BE76B0F
:1017D000E06BE16B120049D8040EE7CFDBFF12008B
:1017E00044D8060EE7CFDBFF1200FD0EDBCFD3F2AD
:1017F000FE0EDBCFD4F21200000EF722F822080012
:10180000F550E66E120000011624146E000E17202B
:10181000156E1200CD90CF6ACE6ACD801200F36EA5
:10182000080EF3CFDBFF1200F36E070EF3CFDBFFE2
:101830001200FD0EDBCFE9FFFE0EDBCFEAFF120048
:10184000020DD950F324E96EDA50F420EA6E12004A
:1018500002013CDF0001E851EE26E951ED221200C1
:10186000DBCFF4FFF350F45C1200DB50300FE76E77
:101870001200E7CFDBFF0A0E2CDF05C0DBFF1200F2
:10188000020124DFEE2A000EEF2212002BDFE652C7
:10189000DF6A0201D2511200CFC2D7F231DFDF6E10
:1018A00000011200010EE3DEEF501200E0DEE5520F
:0418B000E7501200EB
:0C18B4009DD9F2A4FED7D8D903E02A0E7B
:1018C000BB6E01D0BB6A99D133DADF5000080AE25F
:1018D000FE0EDBAE03D0010EE66E01D0E66AEADF53
:1018E000BCD9F3D7E55289D183D9E652080EDF6E11
:1018F000DF50000811E2FE0EDBAE06D0010EE66EF0
:10190000D9DFE552E66A05D0E66AD4DFE552010E7A
:10191000E66ED0DFA2D9ECD7E5526FD169D99492A7
:10192000530ECB6EC40ED56E590ED66EF2942A0E9F
:10193000BB6E070EE66EF80ED2D9080EE66E950E57
:10194000CED9000E0001E76EFD19E8AE02D0FD35DC
:1019500003D0E750D880FD5505E2FD6B040EE66E1E
:10196000300E05D0010EFD6F040EE66EC00EB7D925
:10197000FE0EDBCFE6FFB8DFE552FD0EDBCFE6FF64
:10198000B3DFE552E66A96DFE552948236D130D96C
:10199000F2A4FED76BD903E02A0EBB6E01D0BB6A5E
:1019A0002CD1C6D9DF50000811E2FE0EDBAE06D006
:1019B000E66AEDDFE552010EE66E05D0010EE66E39
:1019C000E6DFE552E66AE3DF48D9ECD7E55215D108
:1019D0000FD99492530ECB6EC50ED56EFA0ED66EFD
:1019E000F294BB6A000E0001E76EFE19E8AE02D069
:1019F000FE3503D0E750D880FE5505E2FE6B030E9E
:101A0000E66EC00E05D0010EFE6F030EE66EE00E10
:101A1000E66EC7DFE552E552FE0EDB50080DFE0E06
:101A2000F3CFDBFF050EE66EFE0E66D9FD0EDB5032
:101A3000040DFD0EF3CFDBFF060EE66EFD0E5CD946
:101A4000E66AA5DFE5529482D8D0D2D8110EE126FD
:101A500075D90B0EEECFDBFF0C0EEDCFDBFF38D9C7
:101A6000ED1001E0A6D0020EBCD8EECF14F0EFCFFF
:101A700015F0830E1502F3CF15F01402F45015265D
:101A8000070EF3CFDBFF080E15C0DBFFB50EB9D88C
:101A9000070E08C0DBFF080E09C0DBFF070EDBCF17
:101AA00014F0080EDBCF15F01406000E155A145072
:101AB000CB6E020EA6D8090E08C0DBFF0A0E09C0C5
:101AC000DBFFBB6A040E8DD8030EEECFDBFF040EE6
:101AD000EDCFDBFF060E85D8050EEECFDBFF060E41
:101AE000EDCFDBFF94929EA2FED79E92090EDB50B3
:101AF000BB6E040EDF6EDFCF14F010D990D81BE25E
:101B0000640EDF5C02E2BFD801D098D8EDD8D5D8FA
:101B100009E29EA2FED7010EDB06020E01E2DB0601
:101B20009E92F5D7BB5004E1090EDB50BB6E01D08D
:101B3000BB6ADF2AE0D7F2D8D9EC14F007C015F061
:101B4000040E0624DF6EDFCF14F0050EDBCF19F094
:101B5000060EDBCF1AF0030EDB501924176E040EAD
:101B6000DB501A20186E020E086E096A17C00DF0BD
:101B700018C00EF054D81BE2640EDF5C02E283D87A
:101B800001D05CD8B1D899D809E29EA2FED7010E47
:101B9000DB06020E01E2DB069E92F5D7BB5004E1A4
:101BA000090EDB50BB6E01D0BB6ADF2ACCD7948212
:101BB00011D08ED806E1600EED1803E1A3D8AEDE99
:101BC00007D086D807E1500EED1804E19BD800DF5E
:101BD000E552E552110EE15C02E2E16AE552E16E86
:101BE0000CD0E76EABD8E750E926000EEA221200CF
:101BF000D9CFE6FFE1CFD9FF1200E552E7CFD9FFF9
:101C00001200146E156A070EDBCF08F0080EDBCF4A
:101C100009F014C00DF015C00EF010EF15F0D9EC5E
:101C200014F006C015F007C016F0040E1526000EBD
:101C300016221550145C000E16541200FB0EDBCF5A
:101C400014F0FC0EDBCF15F0640EDF5C020D1450B7
:101C5000F324E96E1550F4201200E552FE0EDB501D
:101C6000020DFE0EF3CFDBFFDF061200D650146E1E
:101C7000156AA60E145E000E155A1450D66EF29414
:101C8000FE0EDB501200156ADF34FE0B1536146EA3
:101C9000FD0EDB501424E96EFE0EDB501520120001
:101CA0000F0EEECFDBFF100EEDCFDBFF0F0EDBCF05
:101CB000E6FF0D0EDBCFE6FF1200D950010FE96EF3
:101CC000DACFEAFF000ED880EE54000EED54120079
:101CD000D9500B0FE96EDACFEAFFEE501200E66E34
:101CE000F3DDE552E5521200EA6E010EEECFDBFFA6
:101CF000020EEDCFDBFF1200DBCFE6FF52DEE55236
:101D0000E5521200080E6DDF0D0EEECFDBFF0E0E5A
:101D1000EDCFDBFF0A0E65DF50EF0EF0020E086E0E
:101D2000096A030EDBCF0DF0040EDBCF0EF01200BC
:101D30005FDFE652FD0EDB50DF6E1200FD0EDBCFE3
:0A1D4000E9FFFE0EDBCFEAFF120000
:061D4A00040120511F0BF3
:101D5000010801E012002051600BE842E842E8422D
:101D6000E842E842010801E01200245103E02405A2
:101D700001E012002151230A39E0010A33E0030A8D
:101D800025E0010A1CE0240A31E0070A2FE0010ADD
:101D90002DE0030A0EE0010A01E012004ED9020113
:101DA000E40EF86F020EF96F0101C9930201080EEB
:101DB00017D043D90201E40EFA6F020E05D03DD9C7
:101DC0000201D90EFA6F020EFB6F120036D9020122
:101DD000D90EF86F020EF96F0101C9930201070EC7
:101DE000FC6F12002AD922C4E0F212001200020194
:101DF000D96BC20EDA6F010EDB6FDC6BDD6BDE6B55
:101E0000080EDF6FD26BD16B1A0E726E1E0E736EE0
:101E10000401000E166F050E176F400E146F0401BB
:101E2000196F080E1A6F050E1B6F880E186F0401CC
:101E3000480E1E6F050E1F6F400E1C6F1200D9CF8B
:101E4000E6FFE1CFD9FF0201D16B040118BF30D00A
:101E5000FC0EDBCF14F01951D880145403E2FC0EB1
:101E600019C4DBFF0201D16BFC0EDB50D15D19E21E
:101E7000D151EA6A080FE96E050EEA22EF50E66ECC
:101E8000D151E76EFD0EDBCFE9FFFE0EDBCFEAFF9F
:101E9000E750E926000EEA22E552E750EF6ED12B1B
:101EA000E3D70401400E196F1817187D880E181318
:101EB0000201D151E552E7CFD9FF1200ACD802019F
:101EC000D25114E1DF6AB2D802E115500BE0FD0EE9
:101ED000DBCFE9FFDB2AFE0EDBCFEAFF01E3DB2AE3
:101EE000EF50F1E175D8D86B010ED26F9AD093D82C
:101EF0000201D25115E1DF6A99D802E115500CE0D8
:101F0000FD0EDBCFF6FFDB2AFE0EDBCFF7FF01E392
:101F1000DB2A0800F550F0E15BD8010ED86FD26FD4
:101F200080D079D804011CBF52D0030E0201D25DCB
:101F300001E1D26BD2514BE0020ED25D03E104010C
:101F40001D6B3CD0D2053DE1400E146E156AD75191
:101F5000145C000E155803E2400EDF6E02D0D7C2AB
:101F6000DFFFDFCF1DF4DF50D75DD76F480ED56F91
:101F7000050ED66FD8050AE1DF5011E0D3C2F6FF97
:101F8000D4C2F7FF0800F5503AD8F6D7DF5007E083
:101F9000D3C2E9FFD4C2EAFFEF5031D8F7D702012C
:101FA000D7510FE104011D51146E156A400E14182B
:101FB00005E1155003E10201020E02D00201030EF9
:101FC000D26F400E04011C171C7D880E1C1329D0F3
:101FD000DF50146E156AD950FD0FE96EFF0EDA203E
:101FE000EA6E1450EE5E1550ED5AFD0EDBCFD3F2C3
:101FF000FE0EDBCFD4F2DFCFD7F202011200D5C242
:10200000E9FFD6C2EAFFEF6ED52B000ED623D32B05
:10201000D423DF061200D9CFE6FFE1CFD9FFE65285
:102020001200E552E552E7CFD9FF1200DF2ADF5058
:10203000146E156AFF0E141812000201030EF76FDA
:0220400012008C
:0E2042006C5002E0000E01D0010E00090BE010
:10205000040100513C0BE842E8420D0802E13CEF6C
:1020600010F06EEF10F06C5002E0000E01D0010E87
:10207000040901E042D81200D9CFE6FFE1CFD9FF31
:10208000E6520201F66BF76BFC6BFD6B70EC11F026
:10209000DF6ADF50146E156A010E145C000E1558CD
:1020A0001AE20201F75117E1F76ADF34FE0BF73647
:1020B000F66E110EF626290EF7220900F5CF14F060
:1020C0000800F5CF15F004D015C0FAFF1450F96ED2
:1020D000FBDFDF2ADED799D8E552F6D0020E0201E7
:1020E000F65D09E168D8040100BD02D0C80E01D038
:1020F000880E006F12003EEF11F0040E0101C85D62
:1021000009E122C46EFF6E50000802E2050E01D004
:10211000030EC86F0201F60509E10AD8040104BDE7
:1021200002D0C80E01D0880E046F12003EEF11F0ED
:10213000C4D80201080EFC5D000EFD5905E2FCC288
:10214000DEFFFDC2DDFF03D0080EDE6EDD6A040196
:1021500004930491010EDB500413DFCF05F4000E4D
:10216000DB500201FC5F010EDB50FD5B280EFA6FB5
:10217000040EFB6F0101C9A30CD098D815E0F8C27A
:10218000F6FFF9C2F7FF0800F55080D8F6E2DB064B
:10219000F4D78CD809E0F8C2E9FFF9C2EAFFEF50A2
:1021A00075D8F7E2DB06F5D7020EE15C02E2E16AE0
:1021B000E552E16E89D081D8030E04010015E76E67
:1021C000010EE7CFDBFF01C4DFFFDE500201FC2779
:1021D000DD50FD23280EF86F040EF96F67D80EE06E
:1021E000F8C2E9FFF9C2EAFFEF50FAC2E9FFFBC209
:1021F000EAFFEF6E6DD8F2E2DB06F0D7020EE15C8B
:1022000002E2E16AE552E16E5FD00201F75105E1B9
:1022100045D8840E006F04011DD0040120AF1CD0EE
:102220000201FC510401265D0201FD510401275900
:1022300004E226C4FCF227C4FDF27ADF0201010E9B
:10224000F66F2CD8800E006F0401280E066F040E66
:10225000076FC80E046F10D00201020EF66F040162
:10226000056BC80E046F0401080E016F280E026F83
:10227000040E036FC80E006F6D9812000201F66B1A
:102280000DD8880E006F0401046B1200FAC2E9FF3A
:10229000FBC2EAFFEF6E020168EF11F00401080EC5
:1022A000016F200E026F040E036F1200D9CFE9FFF9
:1022B000DACFEAFFEE50ED101200D9CFE6FFE1CF02
:1022C000D9FF020EE1261200E552E7CFD9FF120036
:1022D000FA2B000EFB23F82BF923DF06010E120068
:1022E00004012051600BE842E842E842E842E8423B
:1022F000000901E012002151070A40E00B0A3EE00C
:10230000070A33E0010A23E00B0A1FE0020A1DE07E
:10231000030A19E0080A10E0010A0CE00F0A08E0BD
:10232000030A01E0120012D90101040EC86F120065
:10233000BFEF11F0F6EF11F009D90201CA0EF86FE4
:10234000010EF96F0CD011EF12F043EF12F002D929
:102350000201F86FF96BCB0EF827010EF92301018A
:10236000C9930201010EFC6F1200F4D8EA6ACB0F88
:10237000E96E010EEA2222C4EFFF12001200800E65
:102380000401205D32E12351030A1FE0010A0AE043
:10239000030A29E1DBD80201460EF86F280EF96F17
:1023A000120E1ED0ADD8070EF626290EBBD8020E8F
:1023B0000201F76AF825F66EF951F7220900F5CF08
:1023C000FCF20A00F5CFFDF20ED09AD80B0EF626DD
:1023D000290EA8D8F8C2F6FFF9C2F7FF0800F55099
:1023E0000201FC6FFD6B0101C9831200AFD80F0E13
:1023F000E66E710EE66E0F0E9DD8010EE66ECB0EE8
:10240000E66E010E97D822C4CAF10401225104E1FC
:102410000101050EC86F12000101060EC86FF7EF2B
:102420000EF00401286B296B040120511F0B020AD6
:102430000FE0030A0BE0010A18E188D804012881A3
:102440000101C9A112D0040128830FD07FD80DD07B
:102450004BD801E0010E5DD8FAC2E9FFEA6EEF50F9
:10246000040B03E00401010E286F0201F7050AE1E5
:102470000201280EF86F040EF96F0101C9930201E1
:10248000020EFC6F1200040122050EE120511F0B09
:1024900000090AE15BD8030E0401215D03E101019B
:1024A000C98102D00101C991040122511CE12051CE
:1024B0001F0B020818E124510F0B000914E014D877
:1024C00001E0010E26D8030E0401215D04E1840E13
:1024D00038D8EF6E120024AF03D033D8EF6A120061
:1024E000880E2FD8EF6E120035D80F0B080DF35061
:1024F000156A000F146E040E15222451800B120071
:1025000025D804012251F66EF76AD890F636F736D0
:102510001200040DF35002011424FA6F000E15206E
:10252000FB6F1200F7220900F5CFF8F20A00F5CF91
:10253000F9F21200E66E54EC13F0E552E552E55262
:102540001200FAC2E9FFFBC2EAFF12000201010E0B
:0C255000F76F1200FBDF040124511200A1
:04255C006DA60CD884
:102560000101C80508E16DBA06D0686A696A698028
:102570006988020EC86F12006D6A696A6D86010172
:10258000010EC86F12006D6A696A0101C86B120002
:10259000C3EF12F00101C85101E112006850040BB1
:1025A00004E06950040B01E03CD86DB212006850A1
:1025B000010B04E06950010B01E054D86850100B86
:1025C00004E06950100B01E024D86850400B04E08F
:1025D0006950400B01E03BD86850200B04E0695083
:1025E000200B01E036D86850020B04E06950020B62
:1025F00001E036D8030E0101C85D01E21200685007
:10260000080B06E06950080B03E021EC10F0689617
:102610001200698468986D82A19AA08A0300A09A2A
:1026200012006D926994689412000101C9A10ED044
:10263000F8DF6D840201080EFE6F070EFF6FFE07C4
:10264000000EFF5BFE51FF11FAE16D941200689CD1
:10265000120070A003D03EEC11F07090689A120046
:10266000689212006A6A686A9F0E6B6E7B0E696ED2
:102670006E6A0F0EE66E710EE66E0F0EE66E14D8E1
:10268000E552E552E552160E706E68A602D06896C5
:10269000FCD76D983EEC11F00101C9910101CA6BA4
:1026A0000101030EC86F1200D9CFE6FFE1CFD9FFB9
:1026B000FD0EDBCFE9FFFE0EDBCFEAFFFC0EDB50A9
:1026C00004E0EE6AFC0EDB06F9D7E552E7CFD9FF4E
:0226D0001200F6
:0E26D200DACFE4FFE9CFE4FFEACFE4FFE652FF
:1026E0009EA45AD00001DDB121D0BD6A060EBD6E98
:1026F0009E94DD81BF501C6E1B6ABE5000011B24DE
:10270000EA6F000E1C20EB6F0001DE6BDF6B9EA0FA
:1027100009D09E900001000ED880EA55010EEB55BD
:1027200001E282D80001E06BE16B41D09E94DD8331
:10273000BF501B6E1C6A1C6E1B6ABE5000011B241E
:10274000E66F000E1C20E76FDEC0E8F0DFC0E9F0A6
:102750009EA014D09E9068D80001E65D010EE75956
:1027600004E20001E82B000EE9234CD807E353D81C
:1027700004E30001DD85F29C01D032D80001E02B9A
:10278000000EE1230001ED510001E05D0001EE517A
:102790000001E1590CE306D09E9046D833D807E3F8
:1027A0003AD804E30001DD85F29C01D019D8E55246
:1027B000E5CFEAFFE5CFE9FFE5CFDAFF1100D8CF9B
:1027C000E4FFE0CFE4FFE46EDACFE4FFE652E55247
:1027D000E5CFDAFFE550E5CFE0FFE5CFD8FF100009
:1027E0000001EC5126D8EECFE2F0EDCFE3F0EC297A
:1027F000EC6FE8501ED8EECFE4F0EDCFE5F0EC2919
:10280000EC6F12000001E2510001DE5D0001E351B6
:102810000001DF5912000001E4510001E05D0001F8
:10282000E5510001E15912000001DE2B000EDF230B
:102830001200E96EEA6AD890E936EA36600EE926B7
:06284000000EEA22120066
:0A2846001201000202000008D8048D
:1028500017FE00000102000109024300020100808E
:1028600032090400000102020100052400100104E5
:102870002402020524060001052401000107058247
:102880000308000209040100020A00000007050312
:1028900002400000070583024000000403090434DD
:1028A0000348006F006D006500630069006E0065FD
:1028B000006D0061002D00660072002E0063006F45
:1028C000006D0020002000200020002000200020BB
:1028D000002000340343006F006C006F0072006939
:1028E000006D006500740072006500200048004320
:1028F0000046005200200020002000200020002080
:1029000000200020002000582858289B289F28D30A
:03291000284A1D35
:0C2914002A0EF66E080EF76E000EF86E2C
:1029200002010900F550F16F0900F550F26F03E163
:10293000F16701D03DD00900F550EC6F0900F5506A
:10294000ED6F0900F550EE6F09000900F550E96ED2
:102950000900F550EA6E090009000900F550EF6F13
:102960000900F550F06F09000900F6CFF3F2F7CF38
:10297000F4F2F8CFF5F2ECC2F6FFEDC2F7FFEEC2CB
:10298000F8FF0201EF5302E1F05307E00900F550B0
:10299000EE6EEF07F8E2F007F9D7F3C2F6FFF4C2E4
:1029A000F7FFF5C2F8FF0201F107000EF25BBFD797
:0229B000120013
:0E29B20008C012F008500D02F4CF07F0F3CF6A
:1029C00006F009500E02F4CF09F0F3CF08F00D0223
:1029D000F3500726F4500822E86A092212500E022A
:0E29E000F3500726F4500822E86A0922000C82
:0229EE0004D80B
:1029F0000FD831EC04F0FCD70F0EC112140E6F6E1D
:102A00000101C86B0101C96B0101CA6B1CEF04F025
:102A1000AEEC12F06FBE02D0CAEC12F091EF0FF0E4
:102A2000056A046A100EE76ED89008360936043637
:102A300005360D50045C0E50055805E30D50045E3C
:0C2A40000E50055A082AE72EF0D71200AD
:042A4C00056A080E01
:102A5000E76ED890093605360E50055C02E3056E28
:082A6000092AE72EF7D7120046
:082A680013EE00F023EE00F074
:102A7000F86A019C8AEC14F0F7EC14F0FDD7120010
:102A80000D0076352E34300D0A000D0A003031323B
:042A900030303400AE
:0C2A9400FCFF5C008000B70010006E0129
:102AA00008003803040001050000FE7F2E004000EE
:102AB0005C000800B70004009C01020080020000D6
:102AC000FF3F170020002E0004005C000200CE0033
:102AD000020040010000FF3F170020002E0004000C
:102AE0005C000200CE00020040010000FF1F0C004D
:102AF0001000170002002E00020067000200A00074
:102B00000000909192939495969798999A9B9C9D8A
:020000040030CA
:0100000020DF
:010001000EF0
:0100020038C5
:010003001EDE
:010005008179
:010006008079
:010008000FE8
:01000900C036
:01000A000FE6
:01000B00A054
:01000C000FE4
:01000D0040B2
:00000001FF
